:020000020000FC
:0200000003C03B
:1000060078C00FE50DBF4DE453EC88D00FE107BB78
:10001600002708BB00E800BF00270FBD0DE30EBD9B
:1000260000E409BF05B7006105BF552400E0009351
:100036006000789420916000203069F4C49AC09AD8
:1000460069D0353009F04EC0C09801E000936000D9
:100056005AD0E89447C0213089F45CD0323029F078
:10006600C09A60D0C0985ED03DC0C198052D0230C0
:10007600D4F502E00093600046D034C02230A9F4E3
:10008600C19A48D0323009F02DC0C1980EF006C092
:10009600C398539400E00093600024C0C498C39AA8
:1000A60003E0009360002FD01DC0233059F4C29A9C
:1000B60031D0353009F016C0C29804E000936000D4
:1000C60022D010C0243071F425D0323029F0C29AE3
:1000D60029D0C29827D006C0C29802E000936000DB
:1000E600689411D0A7CF05B7006205BF002708BBEB
:1000F60088950F931F930FB7339511271FBD0FBF19
:100106001F910F91189500B7007F00BF00270FBD04
:10011600302F089500B70F6000BF0895415050403A
:10012600E8F708950F931F931FEF0FEF0A95F1F766
:0A0136001A95D9F71F910F91089553
:00000001FF
